:020000040000FA
:10000000000002286F309A0001309B008030000011
:100010000000122100000000831200009D001B0858
:100020009C0071309E0001309F00831200001C086C
:10003000A0001D08A100FF309C07031C9D032108A0
:10004000200403199A2804301E07A000A101A10D65
:100050001F08A10720089A0021089B00803000009B
:10006000000012210000000083120000A3001B0802
:10007000A2001E089A001F089B00803000000000AC
:1000800012210000000083120000A500A1001B083F
:10009000A000A40002301E07A000A101A10D1F08AE
:1000A000A10720089A0021089B0080300000000072
:1000B00012210000000083120000A100A7001B080D
:1000C000A600A000831200002208A6002308A700B3
:1000D000FF30A207031CA303270826040319932853
:1000E00024089A0025089B0080300000000033217E
:1000F0000000000083120000A600200883120313F2
:1001000084008313831200002118831726088312AA
:100110000313800083120000A40A0319A50AA00A91
:100120000319A10A62280630831200009E070318F3
:100130009F0A1528000000009E280800B501013024
:10014000AF006730AE008030B0002E089A002F0854
:100150009B00300846213508AE00AF0143305E21D8
:100160003A305E21C8302E02031CC02832305E2196
:100170002E08B00038303007AE000130AF00CD2877
:1001800064302E02031CCD2831305E212E08B000D1
:100190009C303007AE000130AF003030B0000A3084
:1001A0002E02031CDA282E08B100F6303107AE000B
:1001B000B00ACF283008B1002F08031DE32830080B
:1001C000303A0319E52831085E212E08AF0030309F
:1001D0002F07AE005E210130AF007730AE008030D7
:1001E000B0002E089A002F089B0030084621B50A5F
:1001F000B201B301B4013408A800280AB4003408DD
:10020000031DFB28330AA800B30028081E3A031D6B
:10021000FA283208A800280AB200743A031DF92807
:10022000AB280800003A03191A29803A0319242937
:100230009B0100341A08840083131B1883170008DD
:100240009B00840A0008080000000000412199007A
:100250009A0F9B039B0A0000000041219800190897
:100260009B0018080800003A03193A29803A03193C
:10027000412900341A08840083131B1883170008CF
:1002800008001B088A001A0882000800AC001B083E
:10029000AB001A08AA002A089A002B089B002C0819
:1002A0003321AD002D0803195D292D085E21AA0A0E
:1002B0000319AB0A0319AC0A4B290800A8008312E2
:1002C0007208A90029185F292808F000080048349E
:1002D00065346C346C346F340D340A3400340134BA
:1002E00000347A34013436340034013400340D34AF
:0602F0000A340034003462
:00000001FF
